:020000040800F2
:1000000000800020A5230008EF230008FD2500083C
:1000100000000000000000000000000000000000E0
:10002000000000000000000000000000AB230008FA
:100030000000000000000000AD2300083514000897
:10004000AF230008B1230008B3230008B52300083C
:10005000B7230008B9230008BB230008BD2300080C
:10006000BF230008C1230008C3230008C5230008DC
:10007000C7230008C9230008CB230008CD230008AC
:10008000CF230008D1230008D3230008D52300087C
:10009000D7230008D9230008DB230008DD2300084C
:1000A000DF230008E1230008E3230008E52300081C
:1000B000E7230008E9230008EB230008ED230008EC
:1000C0004543532E46573A30312E30302E303000D3
:1000D0000120C006014908607047C04608ED00E0F5
:1000E00080B588B03C48006838210840202801903D
:1000F00000D951E00198C046784400794000874417
:100100004B4B4B4B4B4B4B4B104B4B4B4B4B4B4B7A
:100110001E4B4B4B4B4B4B4B144B4B4B4B4B4B4B93
:10012000190031482F49016045E02F487D2109021F
:10013000016040E02C480121C90301603BE02748F1
:1001400001680322114004910068702108400009F1
:10015000401C03900498032805D10399214802F01C
:1001600055FA069004E003991D4802F04FFA0690F4
:1001700006981A490A687F231B021A40120A424352
:1001800006920868400F401C05900698059902F0F9
:100190003DFA154908600EE0144800680721C902BD
:1001A0000840C00A01218140029102990C4802F0E6
:1001B0002DFA0D490860084800680F21090208401F
:1001C00080090B4908580790079807490A68C240F8
:1001D0000A6008B080BDC046081002400C10024002
:1001E0000024F40000127A000000002000100240F9
:0401F000F40100080E
:1001F40000000000000000000000000000000000FB
:1002040000000000000000000000000000000000EA
:1002140001000000020000000300000004000000D0
:1002240006000000070000000800000009000000AC
:10023400F0B503AFFFB0C2B06E46FB4989197163D4
:10024400FA488019B062FA488019F062F01D313022
:1002540030630020086100F0D3FD716BFA48006838
:10026400C860FA48FA4901F09DFDFA4800F01CFF05
:100274000146F94880190180008800B2401C00281A
:1002840012D1F648F64901F08DFD716BEE48006815
:10029400C968401AF349884205D300F0A5FF716B81
:1002A400E9480068C860DCE7EB488019008800B2C0
:1002B400801C002806D1EC48E54901F073FD00F0EC
:1002C40093FFCEE7E4488019008800B27F2817D056
:1002D400E1488019008802B2E448E1497F2301F033
:1002E40061FD716BD8480068C968401ADD498842CD
:1002F40005D300F079FF716BD3480068C860B0E79C
:10030400DB48D34901F04EFD02F062F9D94800F010
:10031400CBFE0146D84880190180008800B2801CB9
:10032400002801D100F025FDD3488019008800B2CF
:10033400401C002800D1E9E7CE4800F0B5FE014694
:10034400C04880190180008800B2002800D5DDE78C
:10035400716B4A68C948801902700968C943C84A60
:1003640092191170007802281FD1C54880190078AD
:1003740002281AD1C348B64901F014FDB26AC24832
:1003840080197921017001234370C04BD367D36F67
:100394005B780F2423408370D26F1278C27001718E
:1003A400052100F0B1FF00F0E2FCB44880190078A8
:1003B40000286FD1B2488019007800286AD1B44867
:1003C400A34901F0EFFCB26AB24B9B1933620025DA
:1003D4001D701C78B0488019706279210155926EA5
:1003E400521C1A70D2B20B248454B26A926E521CFC
:1003F4001A70D2B211248454B26A926E521C1A70CA
:10040400D2B28554B26A926E521C1A70D2B20125CD
:100414008554B26A926E521C1A70D2B20225855467
:10042400B26A956E6D1C1D70EDB24455946E641CD9
:100434001C70E5B221244455946E641C1C70E5B212
:1004440031244455946E641C1C70E5B24324445515
:10045400946E641C1C70E5B263244455946E641C51
:100464001C70E5B273244455946E641C1C70E5B290
:1004740082244455946E641C1C70E5B29224445545
:10048400926E521C1A70D2B281540F2100F03CFFBC
:1004940000F06DFC794880190078112800D00BE138
:1004A400774880190078112800D005E17B48684915
:1004B40001F078FC02F08CF8B16A00200866784AF2
:1004C4001071D0709070507010708865B06A806D33
:1004D400042818DC674800F0E7FD014671488019DC
:1004E4000180008800B2002803D5B16A01200866A3
:1004F40009E0B16AC86D8A6D69498854B16A886D2A
:10050400401C8865E2E7B06A006E002800D0FDE672
:10051400726B6349F1610B784878434088784340B3
:10052400C87843406048801903700C784B781B02EC
:100534001C198D78CB781B025B191B041B19936162
:1005440093691BBA53615269130ECB70130C8B70F1
:100554000A70120A4A700078097988426AD15048B0
:1005640002784178090289188278C07800028018DC
:10057400000442184D48364901F014FC02F028F8F2
:10058400B16A00200866C864B06AC06C012819DC2E
:10059400384800F089FD01464248801901800088EE
:1005A40000B2002803D5B16A012008660AE0B16AE6
:1005B400C86DCA6C3E4989198854B16AC86C401C1C
:1005C400C864E1E7B06A006E002800D09EE63849AE
:1005D40089194878C043487008784978884220D1FE
:1005E40001F0F6FFB36A3249891971610C78621C13
:1005F400684698640834072084436846001BB06149
:1006040085465A640978491CEC2202F012F8716993
:10061400B0690978491C00F077FEB06A806C8546A1
:1006240001E001F0DFFF0BE0DC0200004C020000FF
:10063400400100001F480A4901F0B4FB01F0D2FF59
:1006440095E3C046DC02000080000020882B0008EF
:10065400BC2B000810270000E40200009B2A0008BD
:10066400C42B000811270000CC2B0008E02B000845
:10067400E026000888130000E0020000D802000011
:10068400D4020000F3260008CC0200000058014008
:10069400142C0008B4020000B8020000282C000842
:1006A40048050020A8020000A00200000B29000851
:1006B4009C02000029290008F348801900780128C9
:1006C40012D1F2488019007801280DD1F048801920
:1006D400792101701122427000228270C27001716E
:1006E400052100F011FE42E3E74880190078432811
:1006F40000D00DE1E54880190078432800D007E1D7
:10070400E448E54901F04EFB01F062FFE34800F0E4
:10071400CBFC0146E24880190180008800B2002821
:1007240000D5F3E5B16ADE488019008803B2981C4D
:100734006A464A630933072293436A46D21A3261EE
:10074400954608630020C8624862B06A406AD4498A
:100754008919098809B2891C884218DACF4800F03F
:10076400A3FC0146CF4880190180008800B200280C
:1007740003D5B16A0120C86209E03169B26A906A9E
:10078400526A8854B16A486A401C4862DDE7B06A1C
:10079400C06A002803D0B16A04200862B0E0C048EF
:1007A4008019008800B2411CBF4801F0FBFAB16A0D
:1007B400886BBE4A9219107000208861B06A806903
:1007C400B7498919098809B2491C884212DA306983
:1007D400B16A8A69835CCA695A40B44B9B191A701E
:1007E4008969415CB24801F0DDFAB16A8869401C4C
:1007F4008861E3E7AF4801F0D5FA3269AB48801964
:100804000078A7498919098809B289184978884262
:1008140071D1A9480068C00F002804D0A749A8488E
:100824000860A8480860A8489B4901F0BBFAB16A6F
:1008340000204861B06A406999498919098809B258
:10084400491C88424ADA3069B16A4969405C062821
:100854003FDB9E480068C003002804D59C488E49AD
:1008640001F0A0FAF5E73069B26A984B196819608B
:100874009149F1600B683F24E400A3430B60526983
:10088400805CC200086810430860086802221043B4
:100894000860086801221204104308608B4800684D
:1008A400C003002808D53069B16A4969425C8948A7
:1008B400794901F077FAF1E73069B16A4969425C34
:1008C4008548754901F06EFA7B4908680222904315
:1008D4000860B16A4869401C4861ABE77F486E49CB
:1008E40001F060FA744908680122D20710430860D5
:1008F40001F06EFE01E001F075FEB16A00200862AD
:10090400B06A416B8D46006A002800D0FEE42EE2F6
:100914005D4880190078312800D010E25B488019C6
:100924000078312800D00AE26D485B4901F03AFAB8
:1009340001F04EFEB16A002008616A4A1071D0705D
:100944009070507010708860B06A8068042818DC59
:10095400524800F0A9FB01466348801901800088D1
:1009640000B2002803D5B16A0120086109E0B16A28
:10097400C8688A685B498854B16A8868401C886082
:10098400E2E7B06A0069002800D0BFE455490A785C
:100994004878424088784240C8784240F6488019F6
:1009A400027000780979884200D0C5E101F010FE98
:1009B400F74800F079FB0146F0488019018000886F
:1009C40000B2002800D5A1E4EC488019008800B2E8
:1009D400401C810F411803229143401A002806D07D
:1009E400E748ED4901F0DEF901F0FCFDA3E1012047
:1009F4000102E4488019FF2201F01BFEB26AF16A89
:100A0400002010614860F06A4068F8498919098833
:100A140009B2491C88421ADADD4800F045FB014658
:100A2400F44880190180008800B2002803D5B16A17
:100A3400012008610BE0F16AB06AC0684A68EF49B6
:100A440089198854F16A4868401C4860DBE7D54836
:100A540000684007002803D5D4490420086002E058
:100A6400D14904200860B06A0069002800D04DE430
:100A7400C74800F019FB0146DE4880190180008850
:100A840000B2002832D541E4D8020000D4020000AC
:100A94008802000047290008BC2B000888130000C6
:100AA40084020000740200000A27000868020000A3
:100AB400442C00085D29000814200240082002404C
:100AC40023016745AB89EFCD1D27000810200240A4
:100AD40034270008C42A00085F2900087D2900087B
:100AE400ED2A00084805002058020000F16AB06AA7
:100AF4000068C14A9219107000200860F06A00680A
:100B0400BA498919098809B2491C88420FDAB06ABE
:100B1400F16A0A68B9498919895C40684840B6494C
:100B240089190870F16A0868401C0860E6E7B24851
:100B340080190078AF498919098809B2884200D020
:100B4400F7E0716B9648B060037842781202D318CC
:100B54008478C278120212191204D2180A620A6A3C
:100B640012BACA61C9690A0EC2700A0C8270017095
:100B7400090A417002784178090289188278C0789C
:100B840000028018000440188949884200D2B9E064
:100B9400834802784178090289188278C078000273
:100BA40080180004401891498919098809B240182D
:100BB4008049884200D9A5E001200102F01D3930A6
:100BC40001F036FD89488019008800B2421C7B4838
:100BD4006E4901F0E7F8316B00204860306B4068E3
:100BE40082498919098809B2491C88420FDA306B95
:100BF4004268824880198018F11D39318A187A496F
:100C040000F086FC316B486810304860E6E76C48B9
:100C14000068C00F002804D06A496B4808606B481C
:100C2400086072488019008800B2421C684857491D
:100C340001F0B8F8316B00200860306B00686B4934
:100C44008919098809B2491CC91088424EDA6148D9
:100C54000068C003002804D562484C4901F0A2F89A
:100C6400F5E7316B5B4A106810604D4803784278B1
:100C74001202D2188378C0780002C01800048018C9
:100C84000968CB00C018F21D3932D118D2584B680C
:100C940000F07EFB4F480068C003002804D550488C
:100CA4003A4901F07FF8F5E74A4800680020002837
:100CB40004D04A48384901F075F812E0316B3848DD
:100CC400037842781202D2188378C0780002C018E0
:100CD400000480180968C90042183F482B4901F0F4
:100CE40061F8316B0868401C0860A6E7344908685D
:100CF4000122904308600868D2071043086001F09D
:100D040067FC15E026480278417809028918827840
:100D1400C078000280180004421834488019008802
:100D240000B2431C24481C4901F03CF801F050FC7B
:100D340001E001F057FC01E001F054FC17E02C48FD
:100D4400801902781348144901F02CF801F04AFC88
:100D5400716B0D480068C968401A1049884206D36F
:100D640000F042FA716B08480068C86001E0FFF7C0
:100D7400CDFAFFF776FAC046500200004C0200009C
:100D8400482C00084801000080000020BC2B00080B
:100D940088130000B5270008C42B000811270000A1
:100DA40048050020140C0050180C0050280C00506A
:100DB40000300008FFEF0108D72900089729000830
:100DC400142002400820024023016745AB89EFCD7F
:100DD400B1290008102002407A2700085F27000884
:100DE400702C000834270008782B00084C020000FF
:100DF400D802000058020000500200004801000020
:100E040010B588B0874800687D21C90001F0FCFB5B
:100E140000F016FB844800F0C5FF84488449854AE5
:100E240000F0C0FF84480068C005002804D5854848
:100E34007F4900F0B7FF09E08048814900F0B2FF24
:100E44007D2080000021C94300F0CAFA7A48006876
:100E54004005002803D57E4800F0A4FF09E0764849
:100E640000684005002804D47748784900F09AFFC8
:100E7400F5E778480068C0B2AA2804D0754800682D
:100E8400C0B2CC283ED1744800688004002839D50B
:100E940072480068C00F002804D071497148086086
:100EA400714808606D4800684000002804D56F4907
:100EB4006F4808606F48086066490868FF229043DD
:100EC40008600868EC22104308606B480068C0039F
:100ED400002800D5F9E7614908680122520410434B
:100EE400086065480068C003002800D5F9E75B493D
:100EF40008680122D206104308600020C143642020
:100F040000F06EFA5D4908680B2210430860052062
:100F140001070868CF2292049043086008684522BC
:100F2400D20410430860564908680322120590430E
:100F340008600868012203921305184308605149A8
:100F4400049108680F242302984308600868130278
:100F5400184308600868F023984308600868102361
:100F64001843086008682404A0430860086814044F
:100F7400204308604449059108683024A043086070
:100F84000868C024A043086008681843086008681B
:100F94004023184308603D490868940320430860CF
:100FA4003B49069108689043086008681307984312
:100FB400086008681303184308600868D30398435B
:100FC4000860086893021843086008680C231843F3
:100FD400086008682F4B184308602F4B186820439B
:100FE40018602E4B2E4818600868104308600020D3
:100FF40007900798042812DC2A490191042008600C
:101004009620029000F0DAF9019A029801218904ED
:10101400116000F0D3F90798401C0790E9E708B085
:1010240010BDC046000000204F2B0008C82C00084B
:10103400BC2B0008C000000800100240712A000800
:10104400C42B0008542B0008E02C0008002D0008D5
:10105400EF27000820200240100000501420024016
:101064000820024023016745AB89EFCD0C200240E4
:101074003B2A19087F6E5D4C102002403410024058
:101084000C00005024000050000C0050401002409E
:10109400003801400000FF03083801400C380140CB
:0810A40041030000180C00508C
:1010AC0080B586B0049040480168039100680290B6
:1010BC003E480068800600281DD43B480068029911
:1010CC00401A0499884200D315E037480068039908
:1010DC00401A4B280ED334480068039034480068FB
:1010EC004007002803D534490420086002E0314948
:1010FC0004200860DCE72C4800680299401A049927
:10110C00884203D305A93548088048E02748006881
:10111C00000700280ED530482A4900F03FFE2A4926
:10112C000820086025480068C0B2019005A927482E
:10113C00088034E01D480068400700280AD525487F
:10114C00204900F02BFE20490420086005A91F4807
:10115C00088024E015480068800700280AD51C4840
:10116C00184900F01BFE18490220086005A9174811
:10117C00088014E00D480068C00700280AD0104809
:10118C00104900F00BFE10490120086005A90F481A
:10119C00088004E009480068C0B205A9088005A8C9
:1011AC00008800B206B080BD800000201C380140D1
:1011BC00140C0050180C0050280C0050243801401E
:1011CC00322B0008C42B000820380140FFFF000020
:1011DC00AC2C00085B2A00083D2A0008FEFF00002A
:1011EC0080B586B0334908680122130318430860A0
:1011FC0031490868104308603048314900F0CEFD91
:10120C000020029002982F49884215D8029839493B
:10121C000091421839482A4900F0C0FD0099029803
:10122C0040580490049800BA039003982849086029
:10123C000298001D0290E5E72348214900F0AEFD1D
:10124C00224800680190224800680199884227D101
:10125C0023481B4900F0A2FD7D20800000F0AAF875
:10126C001449086801221203904308601D490020AC
:10127C0008601D4908601D49086072B61C491D486C
:10128C00086000680590059880F3088862B61A48D3
:10129C00006880470020C1437D2000F09DF8F9E7ED
:1012AC000C480D4900F07AFDFA200C4900F094F836
:1012BC0006B080BD3810024008300240D02700082C
:1012CC00BC2B0008FBBF01001F2B0008FCEF010822
:1012DC0000300240192A0008C42B000888130000B3
:1012EC00982C000818E000E014E000E010E000E0AA
:1012FC0008ED00E000300008043000080A2B00085C
:10130C0080B584B00390029128200190029A17486E
:10131C00174900F043FD0020009000980299884284
:10132C0017DA164800680006002800D4F9E703987D
:10133C000099405C124908600098282805DC039845
:10134C000099415C0F4800F029FD0098401C00906A
:10135C00E3E70298292803DB074800F01FFD02E0B1
:10136C00044800F01BFD04B080BDC046272A0008CD
:10137C00BC2B00085D2900082D2B00081C380140EF
:08138C0028380140282B00085D
:1013940084B0039001930092074908680122104326
:1013A4000860009803990860BFF36F8F0198039950
:0C13B400486004B07047C046142002409E
:1013C00082B00190064800680090054800680099C6
:1013D000401A0199884200D2F7E702B07047C04630
:0413E0008000002069
:1013E40080B584B003900291012080040E49086006
:1013F4000E48006801900D4800680199401A02994E
:1014040088420ED208490091082008600398FFF72B
:10141400D5FF00990120C00408600398FFF7CEFFB0
:10142400E9E704B080BDC046180C005080000020DD
:1014340002490868401C08607047C04680000020CC
:1014440080B584B002900298401E000E002802D09D
:101454000120039010E00298401E09490860002012
:101464000190C043032100F011F801980549086078
:10147400054A072111600390039804B080BDC0465B
:0C14840014E000E018E000E010E000E0E0
:1014900070B582B0024601A802700091007840B297
:1014A000002816D401A9087840B20322D34318407B
:1014B000174A8058097849B28C07E50EFF24AC40E2
:1014C000A043009CA401E4B2AC40204319408850E2
:1014D00019E001A908780F24204008380322D343DB
:1014E00018400A4A8058097849B28D07EE0EFF2548
:1014F000B540A843009DAD01EDB2B5402843214061
:1015000008391940885002B070BDC0461CED00E09B
:0415100000E400E013
:1015140080B584B00390029101920198039900F080
:101524006BFF01980549086002980549086000F0BE
:1015340009F800F078FF04B080BDC0467C000020AC
:0415440084000020FF
:1015480010B586B000200590059803281CD8484897
:101558000168059A9200895C444B99540168059A80
:101568009200521C895C99540168059A9200921C59
:10157800895C9954006805998900C91C405C5854D5
:101588000598401C0590DFE705982B2869D80020AE
:101598000490049803280DD80598800004994018F1
:1015A800324A8018001F007802AA50540498401C40
:1015B8000490EEE705A800788007002828D102A843
:1015C800017803914178017081784170C178817008
:1015D8000399C17001780190084600F04BF8019911
:1015E8000870487800F046F801994870887800F04B
:1015F80041F801998870C87800F03CF80199C870E2
:101608000298059A9208184B9A5C50400870FFE7B8
:101618000598164980000A18103A1278029B5A4019
:101628000A5405988000401802460F3A127802AB17
:101638005C786240427005988000401802460E3A75
:1016480012789C78624082700598800040180146A4
:101658000D390978DA785140C1700598401C059019
:1016680092E706B010BDC046FE2700088804002097
:0416780084000020CA
:10167C0081B001466A4610701078024A105C01B0C5
:08168C007047C046082D00085C
:1016940083B0014602AA107001A80022027001A8BA
:1016A4000078032822DC684600210170684600782F
:1016B400032816DC02A80078000101A90978890032
:1016C40040186A4612788018094B185C094B1B684D
:1016D40059188B5C43408B540098401C6946087031
:1016E400E4E70198401C01A90870D8E703B07047EB
:0816F400880400207C000020A6
:1016FC0081B01A480168497B6A46117001684B7ABF
:10170C004B7301684B794B7201684B784B710099A4
:10171C000368597001688978117001688B7A8B7035
:10172C0000990368997201688979117001688B7B43
:10173C008B710099036899730168C97811700168FD
:10174C00CA79CA700168CA7ACA710168CA7BCA723E
:10175C0000990068C17301B07047C0467C0000203E
:10176C00B0B586B005A80021017005A80078032843
:10177C0028DC04A80021017004A8007803281CDCD4
:10178C001148016804AA13789B00C91805AB1C7892
:10179C00095D039008460292019300F0F3FA039955
:1017AC000A68029B1C78A4001219019C25785055DC
:1017BC000498401C04A90870DEE70598401C05A994
:0C17CC000870D2E706B0B0BD7C00002021
:1017D800B0B5DEB000205D905D98032800DDD1E251
:1017E800FC4801685D9A9200895C5CAA11700168E6
:1017F8005D9B9B00C91849785BAB197001685D9CBB
:10180800A400091989785AAC217001685D9DAD0062
:101818004919C97859AD29701178589008465792D6
:1018280056935594549500F025FE57990A7853908D
:10183800104600F01FFE00F01DFE539941405798D6
:101848000078529100F016FE00F014FE00F012FE2F
:101858005299414057980078519100F00BFE00F0E2
:1018680009FE00F007FE00F005FE56990A78509030
:1018780010464F9200F0FEFD4F994140569800786F
:101888004E9100F0F7FD00F0F5FD56990A784D905D
:10189800104600F0EFFD00F0EDFD00F0EBFD4E9975
:1018A8004140569800784C9100F0E4FD00F0E2FDCC
:1018B80000F0E0FD00F0DEFD51994C9A5140559A38
:1018C80013784B9018464A91499300F0D3FD5599E7
:1018D8000A784890104600F0CDFD00F0CBFD4999FC
:1018E800414055980078479100F0C4FD00F0C2FDD2
:1018F80000F0C0FD4799414055980078469100F0A6
:10190800B9FD00F0B7FD00F0B5FD00F0B3FD4A9950
:10191800469A5140549A13784590184644914393F7
:1019280000F0A8FD54990A784290104600F0A2FDF4
:1019380000F0A0FD54990A784190104600F09AFDF5
:1019480000F098FD00F096FD4399414054980078C6
:10195800409100F08FFD00F08DFD00F08BFD00F050
:1019680089FD4499409A5140589A13685D9CA40097
:10197800195557990B783F9018463E9300F07AFD19
:1019880057990A783D90104600F074FD00F072FDFA
:1019980057990A783C90104600F06CFD00F06AFDFB
:1019A80000F068FD3E994140579800783B9100F05F
:1019B80061FD00F05FFD00F05DFD00F05BFD5699F4
:1019C8000A783A90104600F055FD56990A783990F1
:1019D800104600F04FFD00F04DFD399941405698F2
:1019E8000078389100F046FD00F044FD00F042FD1B
:1019F8003899414056980078379100F03BFD00F047
:101A080039FD00F037FD00F035FD3B99379A51401C
:101A1800559A1378369018463591349300F02AFD7C
:101A28003499414055980078339100F023FD00F037
:101A380021FD55990A783290104600F01BFD00F000
:101A480019FD00F017FD3399414055980078319100
:101A580000F010FD00F00EFD00F00CFD00F00AFD96
:101A68003599319A5140549A1378309018462F91ED
:101A78002E9300F0FFFC54990A782D90104600F040
:101A8800F9FC00F0F7FC2E994140549800782C910D
:101A980000F0F0FC00F0EEFC00F0ECFC2C9941406A
:101AA800549800782B9100F0E5FC00F0E3FC00F07E
:101AB800E1FC00F0DFFC2F992B9A5140589A1368EB
:101AC8005D9CA4001B19597057990B782A901846E9
:101AD800299300F0CFFC57990A782890104600F017
:101AE800C9FC00F0C7FC2999414057980078279114
:101AF80000F0C0FC00F0BEFC00F0BCFC279941409F
:101B080057980078269100F0B5FC00F0B3FC00F07F
:101B1800B1FC00F0AFFC56990A7825901046249243
:101B280000F0A8FC56990A782390104600F0A2FC11
:101B380000F0A0FC56990A782290104600F09AFC12
:101B480000F098FC00F096FC2499414056980078E3
:101B5800219100F08FFC00F08DFC00F08BFC00F070
:101B680089FC2699219A5140559A13782090184655
:101B78001F9100F07FFC55990A781E90104600F0DE
:101B880079FC00F077FC1E994140559800781D912A
:101B980000F070FC00F06EFC00F06CFC1D994140F8
:101BA800559800781C9100F065FC00F063FC00F08B
:101BB80061FC00F05FFC1F991C9A5140549A1378FD
:101BC8001B9018461A91199300F054FC199941403A
:101BD80002E0C0467C00002054980078189100F07C
:101BE80049FC00F047FC54990A781790104600F019
:101BF80041FC00F03FFC00F03DFC1899414054982E
:101C08000078169100F036FC00F034FC00F032FC4D
:101C180000F030FC1A99169A5140589A13685D9C46
:101C2800A4001B19997057990B78159018461493AE
:101C380000F020FC1499414057980078139100F067
:101C480019FC00F017FC57990A781290104600F01A
:101C580011FC00F00FFC00F00DFC1399414057985F
:101C68000078119100F006FC00F004FC00F002FC82
:101C780000F000FC56990A78109010460F9200F078
:101C8800F9FB56990A780E90104600F0F3FB00F025
:101C9800F1FB0F994140569800780D9100F0EAFB4E
:101CA80000F0E8FB00F0E6FB0D99414056980078FB
:101CB8000C9100F0DFFB00F0DDFB00F0DBFB00F037
:101CC800D9FB11990C9A5140559A13780B901846E4
:101CD8000A91099300F0CEFB55990A7808901046AE
:101CE80000F0C8FB00F0C6FB55990A78079010462B
:101CF80000F0C0FB00F0BEFB00F0BCFB09994140BE
:101D080055980078069100F0B5FB00F0B3FB00F0A1
:101D1800B1FB00F0AFFB0A99069A5140549A137828
:101D280005901846049100F0A5FB54990A78039091
:101D3800104600F09FFB00F09DFB0399414054982A
:101D48000078029100F096FB00F094FB00F092FB03
:101D58000299414054980078019100F08BFB00F003
:101D680089FB00F087FB00F085FB0499019A51403C
:101D7800589A13685D9CA4001B19D9705D98401C83
:081D88005D9029E55EB0B0BDDD
:101D900081B001466A4610701078024A105C01B0AA
:081DA0007047C046082E000840
:101DA80083B0B0B599B004461DA80EC01DA8009018
:101DB80001AD284600F08AFC4020079028462030D4
:101DC80005900748089007480290009A284621463F
:101DD80000F08CF819B0B0BC02BC03B00847C0468C
:081DE800C1240008FFFFFF7F8A
:101DF00070B5114C0020A0621049114A0223102531
:101E0000104EA264E6642565E062A065E0650125E8
:101E1000AD0223616361A261E16125626062606578
:101E2000E01D094900F037FB0849204600F033FB6C
:101E30002020A07170BDC046040000208800002052
:101E4000692B000838050020082F0008FD2800082D
:101E5000F0B581B014460D46182141431648461886
:101E6000F06A1836022810D0012815D00027002863
:101E70001ED1304600F02BFBA04219D33046294634
:101E8000224600F02FFB274612E030462946224624
:101E900000F0E4FB07460BE0304600F018FB074675
:101EA000A04200D32746304629463A4600F01AFBA6
:0C1EB000384601B0F0BDC0460400002020
:101EBC00F0B581B014460D4606460A480078002855
:101ECC0001D1FFF78FFFEFF31087012181F3108809
:101EDC00304629462246FFF7B5FF87F3108801B03C
:081EEC00F0BDC0460400002017
:101EF400F0B593B007920F4606460021016010A882
:101F0400401E0D9001200202059242020C924203EF
:101F14000092820301920290C0030B900391CC4380
:101F24000E960F943978252907D0002900D10EE2A6
:101F34007F1C304600F0F1FAF4E7FF1C039DE11921
:101F4400481E00780346203B102B29D880229B0092
:101F540001A4E3580F9C9F46A11F0008C31F00085B
:101F6400C31F0008BD1F0008C31F0008C31F0008CB
:101F7400C31F0008AF1F0008C31F0008C31F0008C9
:101F8400E11F0008B31F0008C31F0008B71F0008A3
:101F9400C31F0008C31F0008BB1F000840220BE03A
:101FA4005E280CD10120020306E00B9A04E02022F3
:101FB40002E0102200E00C9A15437F1CBFE70023C7
:101FC4000246303A092A06D80A225A438318303B7B
:101FD4000878491CF4E708930F460BE0079802C8F9
:101FE4000790002901D510200543385DCA178918C8
:101FF400514008912E280CD138782A2833D178788A
:10200400BF1C079A02CA0792002903DB059A1543ED
:1020140000E00021089AD217682831D07A2801D02C
:10202400742801D138787F1C089B93430893024697
:10203400633A152A2CD8C0467A4412795200974440
:10204400330B0A0A0A0A0B0A0A0A0A424A590A0AFA
:10205400660A770A0A8665E7019E354300220692DE
:102064002A46079C85E07F1C00210246303A092A53
:10207400CAD80A224A438118303938787F1CF4E7D9
:10208400387868280CD1082005437878BF1CCBE742
:10209400252858D0582858D0002800D042E766E1B7
:1020A4007F1C04231D43BFE7079C26780898421E23
:1020B4000E9829460A9200F080FA0E983146064698
:1020C40000F02BFA37E1280700D516E13068079AAB
:1020D4001168086015E1059A15422A4602D02A467D
:1020E400A64B1A402B06DB1730241C400694079C91
:1020F400019E3EE0280605990D43C01723210140A7
:102104000691079808C8079008200490A4E007984F
:10211400006800289C4E00D006462C469748044090
:102124000598054200D0EFE0304600F0B9F9EEE042
:10213400059A154201D0914A15402A46079C019EF2
:102144000023069315E02521F3E6009A15438A4BF4
:10215400782800D12033079C019E2A06D2170692C4
:10216400059A154201D0854A15402A46069D1D4010
:1021740006950423134007942468324205D1002BAA
:1021840009D1130717D5E4B215E0002B05D11307C5
:1021940004D5E4B204E0A4B20DE024B2002C07D4C8
:1021A400930603D4530606D5202303E02B2301E032
:1021B40064422D230693059B1A4201D06F4B1A40AB
:1021C4001546059A1542029A234600D00A460492FF
:1021D4000799091D079101466F390026092913D86B
:1021E4007944097949008F4404374B4B4B4B154BC9
:1021F4004B370026002B43D007201840303010A95D
:102204008855DB08761CF5E7582825D0642801D0CA
:10221400692835D129460B98014009910026002BE5
:102224002ED00998002807D003203040032803D17A
:1022340010A82C218155761C0A24184621460A939D
:1022440000F0E2F9034644430A99091B30220A4389
:1022540010A98A55761CE2E7284600990840002612
:10226400002B0DD00F211940002801D0454A00E071
:10227400434A5118097810AA91551B09761CEFE7B7
:10228400069A511E104688410899891BFF2A00D9D5
:10229400491E081A04998B1BD9178B43C21A0C9830
:1022A4000542099304D10E98294600F086F90022CC
:1022B40006980A92010A03D00E9800F02EF90698A7
:1022C40000280E9C03D00146204600F026F9204643
:1022D40029460A9A00F071F930212046099A00F043
:1022E4005FF9741E06DB0D98815D0E9800F015F9F8
:1022F4002646F6E7E8060E9E20E0079A1068316845
:102304000170121D07920DE6304600F09BF9054658
:102314000898421B0E9821460A9200F04EF9002DAF
:1023240006D031780E9800F0F8F8761C6D1EF6E7AA
:1023340025460E9E079C241D0794E8060F9C00D496
:10234400F0E5202130460A9A00F02AF9EAE5F0681F
:10235400002805D006CE083E914201D2039A425489
:10236400304600F0A7F93468204613B0F0BD30467B
:1023740000F0A0F9F8E7C04658300000FFFDFFFF69
:0C2384001C2F00080C2F00080429000882
:10239000034C206804348047FBE7FDF74BFFFEE762
:0423A0002C2F0008D6
:0623A400FDF794FEF2E7D4
:0223AA00FEE74C
:0223AC00FEE74A
:0223AE00FEE748
:0223B000FEE746
:0223B200FEE744
:0223B400FEE742
:0223B600FEE740
:0223B800FEE73E
:0223BA00FEE73C
:0223BC00FEE73A
:0223BE00FEE738
:0223C000FEE736
:0223C200FEE734
:0223C400FEE732
:0223C600FEE730
:0223C800FEE72E
:0223CA00FEE72C
:0223CC00FEE72A
:0223CE00FEE728
:0223D000FEE726
:0223D200FEE724
:0223D400FEE722
:0223D600FEE720
:0223D800FEE71E
:0223DA00FEE71C
:0223DC00FEE71A
:0223DE00FEE718
:0223E000FEE716
:0223E200FEE714
:0223E400FEE712
:0223E600FEE710
:0223E800FEE70E
:0223EA00FEE70C
:0223EC00FEE70A
:0E23EE0080B50020C143FA20FEF7F5FF80BD48
:1023FC0083B0029001916846002101706846007814
:10240C000F280ADC019869460978405C029A5054FE
:0E241C000098401C69460870F0E703B0704756
:10242A0080B582B001A8002101700A2100900846F7
:10243A00FFF72BF909200099087001A800780128F4
:10244A000EDBFFF756F9FFF78CF901A80078FFF7C2
:10245A001CF9FFF7BCF90198401E01A90870ECE7C6
:10246A00FFF747F9FFF77DF90020FFF70EF902B0F1
:02247A0080BD23
:10247C0081B001466A46107010784200C0091B23D7
:0A248C0043435A40D0B201B070473C
:0E24960000228B5C83540132002BFAD1704778
:0E24A400411C02780130002AFBD1401A70471B
:0E24B200002A03D0013A8B5C8354FBD17047A3
:0E24C00010B500242046FFF7F9FC204610BDA1
:1024CE00C2680169914201D9D04302E0D243891812
:0624DE0080680818704739
:1024E400F0B581B0154604464068A268E6688019D4
:1024F400971BAF4204D92A46FFF7D9FF751909E0A3
:102504000E463A46FFF7D3FFF119ED1B60682A46E1
:0A251400FFF7CDFFE56001B0F0BD58
:10251E00B0B582B00446006900280FD00CCC083C40
:10252E009A4233D26269531C63618154A069616916
:10253E0081422BD1204600F0B8F827E0E068002851
:10254E0009D00CCC083C9A4220D2551C9D4200D199
:10255E00002181541AE0A06800280AD00CCC083C57
:10256E009A4213D2551C9D4200D1002192008150F7
:10257E000CE0E569002D09D005CC083C904205D24F
:10258E0001AB1970012220461946A8472068401C4D
:06259E00206002B0B0BD98
:1025A40070B514460D460646012C05DB3046294617
:0A25B400FFF7B3FF641EF7E770BDE8
:1025BE0080B5CB0606D4890501D5302100E0202157
:0625CE00FFF7E9FF80BDEC
:1025D40080B582B001A8792101700121FEF794FE33
:0425E40002B080BD04
:1025E80080B582B001A81F2101700121FEF78AFE83
:0425F80002B080BDF0
:1025FC0080B57D2080000021C943FEF7EDFE80BD33
:10260C000A000FD00300400800E052008242FCD9BF
:10261C00002000E05208934200D39B1A40418A42AA
:08262C00F8D17047002070474F
:1026340000220B0011001A00002A02D0013A815432
:04264400FCD170470E
:1026480002460020814204D0135C002B01D0401CBC
:04265800F8E77047E8
:10265C00F0B583B017460646C56800203369AB4217
:10266C00019003D9EA439C18B06803E0EA439A1836
:10267C00B06814187268401B844200D30446501989
:10268C00BC4200D33C4602912246FFF70CFF651971
:10269C00B068854200D1002502990198F5603F1B76
:0C26AC0009192018002FD9D103B0F0BD8F
:1026B80010B54269002A08D00446C369002B04D02B
:0C26C8002169204698470020606110BD89
:0C26D40080B500212022FFF7AFFF80BD81
:1026E0002573424C20696E697469616C697A65640E
:0326F0002E0A00AF
:1026F3002573476F74204745545F494420636F6DCA
:072703006D616E642E0A00F7
:10270A000945726173696E67202564207061676587
:03271A00733A000F
:10271D00090925735374617274696E67206572615E
:07272D0073696E672E0A00BC
:1027340009257357616974696E6720666F72207228
:10274400656C656173696E67206F6620464C415302
:0B27540048206D656D6F72792E0A0041
:10275F0009257350726F6772616D6D696E67206FB7
:0B276F0066206661696C65642E0A003C
:10277A0009257350726F6772616D6D696E67206F9C
:10278A0066203820627974657320617420616464FC
:10279A0072657373203078253038582070657266F8
:0B27AA006F726D6564206F6B2E0A00DB
:1027B5002573556E6B6E6F776E20636F6D6D616EF1
:0B27C5006420307825303258210A00D3
:1027D00025735374617274696E672063616C6375ED
:0F27E0006C6174696E67204657204352430A00AC
:0F27EF004853492069732072656164792E0A008E
:1027FE008D01020408102040801B366CD8AB4D9A18
:10280E002F5EBC63C697356AD4B37DFAEFC5913996
:10281E0072E4D3BD61C29F254A943366CC831D3AC0
:10282E0074E8CB8D01020408102040801B366CD852
:10283E00AB4D9A2F5EBC63C697356AD4B37DFAEF63
:10284E00C5913972E4D3BD61C29F254A943366CCDB
:10285E00831D3A74E8CB8D01020408102040801BC2
:10286E00366CD8AB4D9A2F5EBC63C697356AD4B31F
:10287E007DFAEFC5913972E4D3BD61C29F254A94AA
:10288E003366CC831D3A74E8CB8D01020408102008
:10289E0040801B366CD8AB4D9A2F5EBC63C6973505
:1028AE006AD4B37DFAEFC5913972E4D3BD61C29F8C
:1028BE00254A943366CC831D3A74E8CB8D0102040D
:1028CE0008102040801B366CD8AB4D9A2F5EBC632F
:1028DE00C697356AD4B37DFAEFC5913972E4D3BD8C
:0F28EE0061C29F254A943366CC831D3A74E8CBB0
:0728FD005345474745520017
:07290400286E756C6C2900C0
:10290B000925734164647265737320307825303800
:0E291B0058207265717565737465642E0A002C
:102929000A2573204D656D6F727920616464726543
:0E293900737320435243206572726F72210047
:102947002573476F7420455241534520636F6D6D62
:06295700616E642E0A000F
:02295D000A006E
:10295F00090925735061676520256420686173201C
:0E296F006265656E206572617365642E0A00F4
:10297D000909257345726173696E67206973206655
:0A298D00696E69736865642E0A0024
:1029970009257344656372797074696E67202564CD
:0A29A7002062797465732E2E2E0055
:1029B1000925735374617274696E672070726F6751
:1029C10072616D6D696E67206F6620256420627982
:0629D1007465732E0A007C
:1029D7002573466F7262696464656E206164647210
:1029E700657373206F662030782530385820666FFE
:1029F700722077726974696E67206F66202564207C
:102A07006279746573207265717565737465642185
:022A17000A00B3
:0E2A19002573435243206572726F72210A00CA
:102A270009257353656E64696E6720256420627992
:062A37007465733A2000F3
:102A3D0025734F76657272756E206572726F722096
:0E2A4D006973206465746563746564210A0012
:102A5B0025734E6F697365206973206465746563B4
:062A6B00746564210A00FD
:102A71002573485349206973206E6F7420747572F1
:102A81006E6564206F6E212050726F6772616D20D8
:0A2A910073746F70706564210A0011
:102A9B0025730A4572726F7220647572696E6720B6
:102AAB0072656365697074696F6E206F66206F6EF7
:092ABB00652062797465210A00AE
:102AC4000909257357616974696E6720666F7220FE
:102AD4007061676520256420746F206265206572CB
:092AE400617365642E2E2E0A00B8
:102AED002573476F74205752495445204D454D4F1E
:0D2AFD00525920636F6D6D616E642E0A00EA
:102B0A000D257309416464726573733A2030782520
:052B1A003038582000D6
:092B1F002573446F6E65210A0064
:052B28002530325800C9
:052B2D002E2E2E0A000F
:102B32002573506172697479206572726F722069AF
:0D2B420073206465746563746564210A0086
:052B4F001B5B324A008F
:102B54002573485349206973207475726E65642027
:052B64006F6E2E0A0057
:092B69005465726D696E616C0027
:042B7400E100000874
:102B78005C383657603D0E38611E4E216219476237
:102B880025730A57616974696E672031307320664E
:102B98006F7220636F6D6D756E69636174696F6EB6
:102BA80020696E697469616C697A6174696F6E2EE7
:042BB8002E2E0A00B3
:082BBC001B5B313B33326D005D
:082BC4001B5B313B33316D0056
:102BCC0025730A54696D656F7574206F66203130FA
:042BDC0073210A0057
:102BE00025730A57726F6E6720494E4954206279E7
:102BF00074652072656365697665642120476F742A
:102C000020257520696E7374656164206F662025C8
:042C100075210A0020
:102C14002573476F742047455420636F6D6D616E53
:042C2400642E0A0010
:102C28002573476F7420524541445F4D454D4F52BF
:0C2C38005920636F6D6D616E642E0A0000
:042C440020256400E3
:102C48000925734279746573206E756D626572200B
:102C58006D757374206279206D756C7469706C651C
:082C6800206F662034210A00F0
:102C700009257357616974696E6720666F722074E5
:102C8000686520656E64206F662070726F67726180
:082C90006D6D696E672E0A00EC
:102C9800257309435243732061726520657175611C
:042CA8006C2E0A0084
:102CAC0025734672616D65206572726F722069734F
:0C2CBC00206465746563746564210A007F
:102CC800257350726F6772616D20737461727465D9
:082CD8006420282573290A007D
:102CE000257357616974696E6720666F7220485357
:102CF0004920746F206265207265616479210A0041
:082D00001B5B323B33336D0015
:102D0800637C777BF26B6FC53001672BFED7AB76A0
:102D1800CA82C97DFA5947F0ADD4A2AF9CA472C04B
:102D2800B7FD9326363FF7CC34A5E5F171D83115B8
:102D380004C723C31896059A071280E2EB27B275D9
:102D480009832C1A1B6E5AA0523BD6B329E32F8451
:102D580053D100ED20FCB15B6ACBBE394A4C58CF49
:102D6800D0EFAAFB434D338545F9027F503C9FA81D
:102D780051A3408F929D38F5BCB6DA2110FFF3D2EB
:102D8800CD0C13EC5F974417C4A77E3D645D19739F
:102D980060814FDC222A908846EEB814DE5E0BDB99
:102DA800E0323A0A4906245CC2D3AC629195E479D0
:102DB800E7C8376D8DD54EA96C56F4EA657AAE082A
:102DC800BA78252E1CA6B4C6E8DD741F4BBD8B8AC5
:102DD800703EB5664803F60E613557B986C11D9E2B
:102DE800E1F8981169D98E949B1E87E9CE5528DFA2
:102DF8008CA1890DBFE6426841992D0FB054BB16CE
:102E080052096AD53036A538BF40A39E81F3D7FB57
:102E18007CE339829B2FFF87348E4344C4DEE9CBA1
:102E2800547B9432A6C2233DEE4C950B42FAC34E16
:102E3800082EA16628D924B2765BA2496D8BD125CC
:102E480072F8F66486689816D4A45CCC5D65B69270
:102E58006C704850FDEDB9DA5E154657A78D9D8414
:102E680090D8AB008CBCD30AF7E45805B8B3450634
:102E7800D02C1E8FCA3F0F02C1AFBD0301138A6B4E
:102E88003A9111414F67DCEA97F2CFCEF0B4E6737E
:102E980096AC7422E7AD3585E2F937E81C75DF6E2C
:102EA80047F11A711D29C5896FB7620EAA18BE1B92
:102EB800FC563E4BC6D279209ADBC0FE78CD5AF438
:102EC8001FDDA8338807C731B11210592780EC5F7E
:102ED80060517FA919B54A0D2DE57A9F93C99CEFDA
:102EE800A0E03B4DAE2AF5B0C8EBBB3C83539961DB
:102EF800172B047EBA77D626E169146355210C7D19
:042F080052545400CB
:102F0C003031323334353637383941424344454613
:102F1C003031323334353637383961626364656643
:102F2C00512F00080400002049050000632F000801
:102F3C00000000204C2F0008040000009B23000818
:042F4C000024F40069
:102F5000206861680834002200E042540139FCD541
:022F60007047B8
:102F620020686168A2680C3401E08B5C8354013AEA
:042F7200FBD57047D4
:04000005080023A527
:00000001FF
